:020000040800F2
:10000000F8250020AD010008B5010008B70100087F
:10001000B9010008BB010008BD0100080000000094
:10002000000000000000000000000000BF01000808
:10003000C101000800000000C3010008AD2700084E
:10004000C7010008C7010008C7010008C701000870
:10005000C7010008C7010008C7010008C701000860
:10006000C7010008C7010008C7010008C701000850
:10007000C7010008C7010008C7010008C701000840
:10008000C7010008C7010008C7010008C701000830
:10009000C7010008C7010008C7010008C701000820
:1000A000C7010008C7010008C7010008C701000810
:1000B000C7010008C7010008C701000801200008A7
:1000C000C7010008C7010008C7010008C7010008F0
:1000D00000F002F800F05AF80AA090E8000C824400
:1000E0008344AAF10107DA4501D100F04FF8AFF2DD
:1000F000090EBAE80F0013F0010F18BFFB1A43F006
:1001000001031847C8490000E84900000A444FF0BD
:10011000000C10F8013B13F0070408BF10F8014B66
:100120001D1108BF10F8015B641E05D010F8016BAB
:10013000641E01F8016BF9D113F0080F1EBF10F80F
:10014000014BAD1C0C1B09D16D1E58BF01F801CB32
:10015000FAD505E014F8016B01F8016B6D1EF9D5B5
:100160009142D6D3704700000023002400250026CA
:10017000103A28BF78C1FBD8520728BF30C148BF0A
:100180000B6070471FB51FBD10B510BD00F01FF903
:100190001146FFF7F7FF03F0A3F800F03DF903B4B1
:1001A000FFF7F2FF03BC00F045F900000948804763
:1001B00009480047FEE7FEE7FEE7FEE7FEE7FEE749
:1001C000FEE7FEE7FEE7FEE704480549054A064B61
:1001D00070470000BD270008D1000008F813002078
:1001E000F8250020F8150020F815002053EA020C2D
:1001F00000F069802DE9F04B4FF00006002B1FBF87
:10020000B3FA83F503FA05F424FA05F65E4012BF4B
:100210001643B2FA82F502FA05F4C5F120051EBFB5
:1002200022FA05FC44EA0C04203556EA044C4FEA55
:10023000144418BF641C4FF000084FF000099042AE
:1002400071EB030C39D3002919BFB1FA81F701FA18
:1002500007F6B0FA80F700FA07F6C7F120071EBFCD
:1002600020FA07FC46EA0C062037B6FBF4FCA7EBA5
:100270000507103F07F01F0BCBF120060CFA0BFB14
:100280002CFA06F644BFB3460026202FA4BF5E46D4
:100290004FF0000B5BEA060C08BF4FF0010B19EBA7
:1002A0000B09ABFB027C48EB0608C01B06FB02CC2B
:1002B0000BFB03CC71EB0C01C1E70B460246414638
:1002C0004846BDE8F08B13B54FF000004FF0000139
:1002D000AFF30080BDE81C407047032A40F2308035
:1002E00010F0030C00F0158011F8013BBCF1020F77
:1002F000624498BF11F801CB00F8013B38BF11F8F8
:10030000013BA2F1040298BF00F801CB38BF00F80E
:10031000013B11F0030300F02580083AC0F008808B
:1003200051F8043B083A51F804CBA0E80810F5E76F
:10033000121D5CBF51F8043B40F8043BAFF3008052
:10034000D20724BF11F8013B11F801CB48BF11F8C7
:10035000012B24BF00F8013B00F801CB48BF00F897
:10036000012B704710B5203AC0F00B80B1E818504F
:10037000203AA0E81850B1E81850A0E81850BFF48F
:10038000F5AF5FEA027C24BFB1E81850A0E818502E
:1003900044BF18C918C0BDE810405FEA827C24BF82
:1003A00051F8043B40F8043B08BF7047D20728BF10
:1003B00031F8023B48BF11F8012B28BF20F8023B5F
:1003C00048BF00F8012B704770477047704775466B
:1003D00000F02CF8AE4605006946534620F00700B1
:1003E000854618B020B5FFF7EFFEBDE820404FF07E
:1003F00000064FF000074FF000084FF0000B21F00F
:100400000701AC46ACE8C009ACE8C009ACE8C009DB
:10041000ACE8C0098D46704710B50446AFF30080C4
:100420002046BDE81040FFF7BABE00000048704704
:100430009813002001491820ABBEFEE726000200F9
:10044000704700002DE9FC410F460478002C00D1D4
:100450000124012502262B484FF09048012C07D09B
:10046000022C20D000243C704FF00110BDE8FC812C
:1004700005700221404602F0C1FE0121404602F013
:10048000BDFE684602F0BCFE00968DF80650694637
:10049000404602F0BFFE00958DF805506946404683
:1004A00002F0B8FEDFE706700221404602F0A6FE29
:1004B0000121404602F0A2FE8021404602F09EFE4D
:1004C000684602F09DFE00968DF80650694640464B
:1004D00002F0A0FE00956946404602F09BFE802097
:1004E00000906946404602F095FE402000900020B2
:1004F0008DF806008DF805506946404602F08AFEE8
:10050000B1E70000541300200278407842EA00204E
:100510004001401EFDD108700048704701000200F4
:1005200070B50446034900250D7001F06FFD25707C
:10053000012070BD5413002030B504464278801C61
:10054000002A0BD010F8013B9D0703D5DB0602D52E
:10055000001D00E0001D521E002AF3D100220A7087
:100560004A70001B0004801C30BD000030B50278CA
:1005700020230E4D4FF09044002A05D0012A0AD0C6
:10058000FF200870284630BD4078C00701D0A36125
:1005900007E0A36205E04078C00701D0A36100E056
:1005A000A36200200870284630BD00000100020050
:1005B00010B503460846002400210522092B1CD053
:1005C00006DC052B34D2DFE803F03333333312007B
:1005D000FC2B2DD004DCF02B15D0F12B28D117E00B
:1005E000FD2B25D0FE2B20D0FF2B21D118E0062497
:1005F00022461049FFF771FE1AE00FA31B68036043
:100600000171144614E033220270417002240FE09D
:100610000170E1214170F5218170C270042407E06E
:10062000402202704170022402E00821017001247E
:10063000204610BD8E4A000856312E3200000000C0
:10064000F0B510F8014B104EB4760022002308E0FC
:1006500010F8015BF7183D7706EB4307BA842A448C
:100660005B1CA342F4D3002006E033181B7FD21A90
:1006700006EB40039A86401CA042F6D30020087087
:10068000641C2004401CF0BD5413002010B50C461F
:100690000E490A78022A14D10078C876897E8842E9
:1006A0000FD20E2000F0CCFF01F0C8F8002121701D
:1006B0006070010AA170010CE170000E2071044805
:1006C00010BDFF2020704FF0011010BD541300200A
:1006D000050001002DE9F047002201F8012B8946B1
:1006E0000125012610F8018B15E010F8017B8246E8
:1006F00007F03F0000B94020C01DC4084A465146DB
:10070000384601F0FDF80AEB040025446D1C39065B
:1007100001D5A1442644B8F10108E6D246EA0540D5
:10072000BDE8F0872DE9F04F85B004460494002021
:10073000029003918D1CD84900220A700026814640
:10074000D64A14F8011BD176927E91427ED214F8DB
:1007500001ABBAF1000F7AD014F8017BF90702D08F
:100760004FF00B0801E04FF00A08B90770D5B9F156
:10077000000F48D0C948B0F810B046450FD1F80670
:100780000DD46946384601F005F902281ED1BBF1A7
:10079000010B1BD3C04909780029F2D016E00A2EBC
:1007A00003D00A26304600F04BFFDFF8EC92694692
:1007B0000E2001F0EFF8022806D1BBF1010B03D3A4
:1007C00099F800100029F2D04FF0000901283ED11D
:1007D000009929700099090A69700099090CA9709B
:1007E0000099090EE9702D1DB9F1000F0BD03906E3
:1007F00009D5AA49896829700A0A6A700A0CAA7080
:10080000090EE9702D1DF90656D520786178E27839
:1008100040EA0120A178090441EA026108430190FD
:10082000241D9E48B0F812B0464503D046463046D7
:1008300000F006FF9948B0F810800021384601F01A
:10084000A9F802280AD1B8F1010802E005E185E023
:100850005DE003D3904909780029EED001287DD1CD
:100860008E48B0F810806946384601F093F80228A7
:1008700006D1B8F1010803D3874909780029F2D0DD
:1008800001280DD18549009A49691140019A914288
:1008900006D0BBF1010B03D37F4909780029DFD0D3
:1008A0007E49009A49691140019A914201D040F075
:1008B0001000012852D18CE0B9F1000F26D1464535
:1008C00003D04646304600F0BBFEDFF8D0B1BBF89F
:1008D00010800021384601F05DF8022806D1B8F1F9
:1008E000010803D36C4909780029F2D001287CD192
:1008F000390609D5DBF8081029700A0A6A700A0C53
:10090000AA70090EE9702D1D4FF0010961E0B9F1DF
:10091000000F27D00A2E03D00A26304600F090FEA2
:100920005E48B0F810B069460E2001F033F8022896
:1009300006D1BBF1010B03D3574909780029F2D046
:10094000012852D1009828700098000A6870009819
:10095000000CA8700098000EE87000E045E02D1D26
:100960004FF0000920786178E27840EA0120A17810
:10097000090441EA026108430090241DB90603D529
:1009800046494861012024E0464503D046463046AA
:1009900000F056FEDFF804B1BBF810806946384617
:1009A00000F0F8FF022806D1B8F1010803D33A4954
:1009B00009780029F2D0012817D1390609D5DBF8CA
:1009C000081029700A0A6A700A0CAA70090EE970E8
:1009D0002D1D0299491C02912F49097829B9AAF1C4
:1009E000010ABAF1000F7FF4B7AEBAF1000F0DD0D3
:1009F00014F8011B8A0703D5C90602D5241D00E09F
:100A0000241DAAF1010ABAF1000FF1D1012834D155
:100A10000A2E02D00A2000F013FEB9F1000F1DD0FB
:100A20001E48068A1C4F69460E2000F0B3FF0228BC
:100A300005D1761E711C02D039780029F3D0012827
:100A40001BD1009929700099090A69700099090C55
:100A5000A9700099090EE9702D1D0EE00F48068A55
:100A60000D4F00210E2000F095FF022805D1761EC3
:100A7000711C02D039780029F3D0DDE9021211701F
:100A8000039948700398291A049805B0201A41EA7E
:100A90000040BDE8F08F0000A002002054130020A9
:100AA0002DE9F84F0446002600208846CF1C524905
:100AB00000220A70DFF844B114F8011B8BF81B10F8
:100AC0009BF81A20914254D22178627841EA02259B
:100AD000A41C002D4DD014F8019B5FEAC97002D010
:100AE0004FF00B0A01E04FF00A0A504600F0A8FD53
:100AF0005FEA89705DD54148048ADFF8FCB00021C7
:100B0000484600F047FF022806D1641E611C03D04E
:100B10009BF800100029F2D0012862D126E03DB9EF
:100B2000BAF10A0F02D00A2000F08AFD4FF00E0938
:100B30003248048A6946484600F02CFF022806D154
:100B4000641E611C03D09BF800100029F2D001281C
:100B500047D1009939700099090A79700099090CF8
:100B6000B9700099090EF9703F1D761C6D1E691C45
:100B7000D5D136E020786178E27840EA0120A1788A
:100B8000090441EA026108430090241D1B48B0F8A3
:100B900010B06946484600F0FDFE022806D1BBF1C0
:100BA000010B03D3144909780029F2D0012818D188
:100BB000761C6D1E681CDDD1BAF10A0F02D00A2026
:100BC00000F03EFD0D48048A0B4D00210E2000F080
:100BD000E1FE022805D1641E611C02D0297800299B
:100BE000F3D088F80060310A88F8011088F8020014
:100BF000A7EB0800BDE8F88FA002002054130020E6
:100C000070B504460D460E492078C876897E884224
:100C100003D3FF202870012070BD082000F010FDD4
:100C20006078A178227940EA0120E178090441EA5C
:100C30000261084301F032F900202870012070BDE4
:100C40005413002010B50278A2F180031F2B02D8A4
:100C500000F06DF810BD01F8012B0C4610F8011BD7
:100C60001E295ED2DFE801F00F171B1F4B4F535DAB
:100C70005723275D5D5D5D5D2B2F33373F43475D18
:100C80005D5D5D5D5D3B0078611CFFF791FC207050
:100C900000F1021010BD2146FFF768FC3EE021463E
:100CA000FFF7D0FB3AE02046FFF73AFC36E021465A
:100CB000FFF72AFC32E0204600F03EF82EE0214605
:100CC00000F030FB2AE0214600F0FAFA26E0214647
:100CD00000F0B2FB22E0214600F034F81EE021468D
:100CE00000F040F81AE02146FFF7F4FC16E0214638
:100CF000FFF7A6FC12E02146FFF7C8FC0EE02146F4
:100D000000F018FC0AE0214600F0DEFB06E0214678
:100D100000F0E8FB02E0214600F022FC00F10110A7
:100D200010BDFF2004F8010C4FF0011010BDFF2092
:100D300008704FF0011070470021417001700220CF
:100D4000704700000078064A00F003035B1C13762E
:100D5000C0F380005076002008704FF001107047FB
:100D6000541300202DE9F05F002201F8012B8A4680
:100D700001254FF0010910F8018B04464FF0904B0C
:100D800033E014F8017B07F03F0000B94020C01D9C
:100D9000C608380606D5DBF8000020F00300CBF8C3
:100DA000000008E00120CBF82800DBF8000040F04C
:100DB0000100CBF8000052462146384601F05EF9AA
:100DC000B8F1000F08D10120CBF82800DBF80000B3
:100DD00040F00100CBF80000380603D56D1CB2448A
:100DE000B14402E0344435446D1CB8F10108C8D266
:100DF00049EA0540BDE8F09F2DE9F04F87B0054670
:100E000006950020049005918C1CDFF850A300216A
:100E10008AF80010002703916D1C15F8018BB8F1BA
:100E2000000F7DD015F8016BB1077AD5F7B3DFF865
:100E300030B3BBF8109006F0110001280DD101A9C4
:100E4000304601F06BF9022815D1B9F1010912D32E
:100E50009AF800100029F2D00DE001A90E2001F04F
:100E60005DF9022806D1B9F1010903D39AF80010FF
:100E70000029F2D00027012852D10199217001994F
:100E8000090A61700199090CA1700199090EE170BC
:100E9000241D5FB131060BD5DBF8081021700A0A5A
:100EA00062700A0CA270090EE17000E000E0241DDF
:100EB000F10651D528786978EA7840EA0120A978C6
:100EC000090441EA0261084302902D1DA448B0F8CC
:100ED00012B0F00711D0A248B0F8109000213046AF
:100EE00001F01CF9022806D1B9F1010903D39AF8DF
:100EF00000100029F2D00128BED19948B0F8109016
:100F000001A9304601F00AF9022806D1B9F1010918
:100F100003D39AF800100029F2D0012810D101E083
:100F200098E069E08E49019A49691140029A91421C
:100F300006D0BBF1010B03D39AF800100029DCD0D6
:100F40008749019A49691140029A914201D040F0C3
:100F5000100001287ED14CE0DFF804B2BBF81090FD
:100F6000F1071DD0F7BB0021304601F0D7F8022869
:100F700006D1B9F1010903D39AF800100029F2D083
:100F8000012867D1310609D5DBF8081021700A0A5B
:100F900062700A0CA270090EE170241D012728E07E
:100FA00001A9304601F0BAF8022806D1B9F10109C9
:100FB00003D39AF800100029F2D001287DD1310620
:100FC00009D5DBF8081021700A0A62700A0CA270B9
:100FD000090EE170241D019921700199090A6170BF
:100FE000019900E005E0090CA1700199090EE1707A
:100FF000241D0021039154E0F7B15948B0F8109036
:1010000001A90E2001F08AF8022806D1B9F10109E0
:1010100003D39AF800100029F2D001284DD101988D
:1010200020700198000A60700198000CA07001986F
:10103000000EE070241D002728786978EA7840EADD
:101040000120A978090441EA0261084301902D1D9D
:10105000B10600E031E003D541494861012020E0BC
:10106000DFF8FCB0BBF8109001A9304601F056F84B
:10107000022806D1B9F1010903D39AF8001000291A
:10108000F2D0012819D1310609D5DBF808102170FA
:101090000A0A62700A0CA270090EE170241D012177
:1010A00003910499491C04919AF8001029B9A8F1F8
:1010B0000108B8F1000F7FF4B5AEB8F1000F0DD004
:1010C00015F8011B8A0703D5C90602D52D1D00E0BE
:1010D0002D1DA8F10108B8F1000FF1D101282FD181
:1010E000EFB11F48068A01A90E2001F017F8022867
:1010F00006D1761E711C03D09AF800100029F2D098
:1011000001281DD1019921700199090A6170019985
:10111000090CA1700199090EE170241D10E00399DA
:1011200071B10F48068A00210E2000F0F7FF022857
:1011300006D1761E711C03D09AF800100029F2D057
:10114000DDE904121170059948700598211A069876
:1011500007B0281A41EA0040BDE8F08FA002002045
:10116000541300202DE9F84F04460026002089463C
:10117000CF1CDFF818A100218AF80010641C217828
:10118000627841EA0225A41C002D74D014F8018B6A
:10119000DFF8FCB05FEA88715BD55FEAC87135D0D3
:1011A000BBF810400021404600F0B8FF022806D1ED
:1011B000641E611C03D09AF800100029F2D00128A7
:1011C00059D123E025B95FEAC87001D04FF00E086D
:1011D000BBF810406946404600F0A0FF022806D147
:1011E000641E611C03D09AF800100029F2D0012877
:1011F00041D1009939700099090A79700099090C58
:10120000B9700099090EF9703F1D761C6D1E691C9E
:10121000D8D130E020786178E27840EA0120A178E6
:10122000090441EA026108430090241D1848B0F8FF
:1012300010B06946404600F071FF022806D1BBF1AC
:10124000010B03D39AF800100029F2D0012812D123
:10125000761C6D1E681CDDD10D48048A00210E200D
:1012600000F05CFF022806D1641E611C03D09AF8CE
:1012700000100029F2D089F80060310A89F80110C5
:1012800089F80200A7EB0900BDE8F88FA002002052
:101290005413002038B50C464178827841EA022286
:1012A000C1780079090441EA00600243009269466E
:1012B000002000F033FF00202070012038BD000026
:1012C00030B50278437842EA03228378C0781B0461
:1012D00043EA006002430F48002A08D00E4D002464
:1012E0000E4BAA4206D301225A705A600FE0FF2229
:1012F0000A7030BD5C700A4D1544B5FBF2F2022A4B
:1013000003D90325B2FBF5F200E001225A600C700C
:1013100030BD00000100040000366E0154130020AF
:10132000FF6BDC02F0B5037842788478C57844EA34
:101330000524057940792D0445EA00600443D5076A
:101340004FF0904006D0DE074FF0020501D08561D6
:1013500000E08562950706D59E074FF0010501D58F
:10136000856100E08562550707D59D08EE074FF0BF
:10137000800501D0856100E08562150607D5DD098D
:10138000EE074FF0100501D0856100E0856200276F
:1013900094B3264DAC4200D92C4664256C43DFF84B
:1013A00090C0DCF80460D50704D00569C5F340059A
:1013B0009D421CD1950705D50569C5F30005B5EB20
:1013C000530F14D1550705D50569C5F3C015B5EB05
:1013D000930F0CD1950602D5B7EB531F07D1150615
:1013E0000AD50569C5F30015B5EBD31F04D0DCF8A9
:1013F0000450AD1BA542D6D30269C2F34002036973
:10140000C3F3000342EA43030269C2F3C01243EA92
:1014100082030269C2F3801243EAC2020069000932
:1014200042EAC01008700348F0BD0000C0C62D009D
:10143000001000E00100060070B50D4610F8014BE9
:101440000146002C01D14FF48074204601F088F948
:1014500000202870E41DE008401C0004401C70BD02
:101460007CB518480021017041700A224260017366
:1014700064220282418241610124047641768176B0
:1014800000F0C4FD684601F0BBFE202500958DF8F4
:1014900006404FF090466946304601F0BBFE00958D
:1014A0006946304601F0B6FE1021304601F0A6FE36
:1014B000102100918DF804406946304601F0AAFEE3
:1014C0007CBD000054130020054A1278012A03D085
:1014D000022A03D0FFF730B8FFF78EBCFFF722B91E
:1014E0005413002010B504461148007801280CD090
:1014F00002280ED000200870487088700320E17820
:1015000089070AD540F4802010BD2046FFF72AFE47
:10151000F5E72046FFF7C4FAF1E76178A27841EADF
:101520000221042202EB810140EA014010BD0000CB
:101530005413002010B5084A037813734378847855
:1015400043EA04231382C378007943EA00205082DF
:1015500000200870014810BD541300200100050050
:1015600010B5094A1278012A07D0022A08D0FF20B4
:101570000870012040F4A02010BDFFF78BFEF9E7B2
:10158000FFF73EFBF6E700005413002070B503465A
:1015900001251878072816D0104C6068A268904280
:1015A00002D16078002810D10D48626800EB8210EB
:1015B0000A461946FEF791FE6068401C606060684C
:1015C000082803D004E00748057070BD0020606063
:1015D0006068A1688842F8D1657070BD740200200F
:1015E000EC050020A002002010B5124C2069E16833
:1015F000884201D1A078D0B10F48216930F811306C
:101600002169A0F5007000EB811281210B4802F0E6
:10161000CCFD2069401C206121690020082900D1EF
:1016200020612169E268914200D1A07010BD0120C3
:10163000207010BD74020020EC090020AC020020D4
:1016400003494978002901D000F004B800F056B8E9
:1016500054130020F0B54FF090420125956102230C
:1016600093629361936293619562936293619362D3
:101670009361802494612049CF7E01EB4706B18CB1
:10168000002904D093629361491E0029FAD11A49B6
:101690001C31795C491E51B1C70701D0946100E04B
:1016A0009462936293614008491E0029F4D1B18E7F
:1016B00091B1C00701D0946100E09462936293619C
:1016C0009461491E21B193629361491E0029FAD1A8
:1016D00095619362936107E09561C00701D09461C1
:1016E00000E0946293629361936293619562936266
:1016F00093619461F0BD0000541300202DE9F04186
:101700004FF090440127A7610226A6624A4B596810
:101710000A46521EFDD1A6610A46521EFDD1A6629E
:101720000A46521EFDD1A6610A46521EFDD1A7628D
:10173000A6620A46521EFDD1A6610A46521EFDD17E
:10174000A6620A46521EFDD1A6610A46521EFDD16E
:101750008025A56193F81B8003EB480CBCF824306E
:1017600053B1A6620A46521EFDD1A6610A46521E18
:10177000FDD15B1E002BF4D12F4A1C3218F8023029
:101780005B1E83B1C20701D0A56100E0A562A6621D
:101790000A46521EFDD1A6610A46521EFDD14008DE
:1017A0005B1E002BEED1BCF8342022B3C00701D061
:1017B000A56100E0A562A6620846401EFDD1A661B3
:1017C0000846401EFDD1A561521E52B1A6620846D0
:1017D000401EFDD1A6610846401EFDD1521E002AC2
:1017E000F4D1A761A6620846401EFDD1A661084655
:1017F000401EFDD10DE0A761C00701D0A56100E04A
:10180000A562A6620846401EFDD1A6610846401E9C
:10181000FDD1A6620846401EFDD1A6610846401EC5
:10182000FDD1A762A6620846401EFDD1A661491EF1
:10183000FDD1A561BDE8F08154130020F0B54FF053
:10184000904301259D6102249C622C4A5168084600
:10185000401EFDD19C610846401EFDD19D629C62E8
:101860000846401EFDD19C610846401EFDD19C6289
:101870000846401EFDD19C610846401EFDD1D27E27
:1018800052B19C620846401EFDD19C610846401E34
:10189000FDD1521E002AF4D100261F229C62084668
:1018A000401EFDD11869C0F380179C610846401E98
:1018B000FDD146EAC7704608521E002AEED19D614E
:1018C0009C620846401EFDD11869C0F380129C61DD
:1018D0000846401EFDD146EAC2709C620A46521E6E
:1018E000FDD19C610A46521EFDD19D629C620A4652
:1018F000521EFDD19C61491EFDD1F0BD5413002044
:101900002DE9F04F00F03F03002B00D140234506A6
:101910004FF001044FF0904802D5C8F8184001E09C
:10192000C8F828404FF0800A4FF00209DFF860B095
:1019300029E011F8016B002708241CE0F50702D00C
:10194000C8F818A001E0C8F828A0C8F82890DBF86B
:1019500004C065466D1EFDD1D8F81050C5F3801542
:10196000C8F81890BCF1010CFCD176087F0847EA52
:10197000C517641E5B1E0CB1002BDFD1E7400406C7
:1019800001D502F8017B002BD3D1BDE8F08F000018
:1019900054130020034A5278002A01D000F004B802
:1019A00000F0FAB8541300202DE9F0474FF09044AE
:1019B0000126A6614FF0020CC4F828C0C4F818C074
:1019C000A662C4F828C0C4F818C0C4F828C0C4F877
:1019D00018C0DFF8BCA19AF81B20002A06D0C4F872
:1019E00028C0C4F818C0521E002AF8D14208D207F5
:1019F0004FF0800501D0A56100E0A562C4F828C0C1
:101A00002269C2F38012C4F818C052008308DB07B1
:101A100001D0A56100E0A562C4F828C02369C3F322
:101A20008013C4F818C01A43C308DB0701D0A561AE
:101A300000E0A562C4F828C02369C3F38013C4F88A
:101A400018C042EA8309B9F1010F05D0A661C4F8B4
:101A500028C0C4F818C07CE04D4B87079A7EDB7E17
:101A6000A2EB03083AD500231F22C4F828C0276937
:101A7000BF09C4F818C043EAC7735B08521E002AA6
:101A8000F3D1A8F10108B8F1000F1AD0C4F828C0AA
:101A90002269C2F38012C4F818C0A8F10108B8F195
:101AA000000F08D0C4F828C0C4F818C0A8F1010875
:101AB000B8F1000FF6D1A661C4F828C0C4F818C068
:101AC00007E0A661C4F828C02269C2F38012C4F8F6
:101AD00018C043EAC27289B30A603AE009681F225B
:101AE000CB0701D0A56100E0A562C4F828C0C4F806
:101AF00018C04908521E002AF2D1A8F10108B8F115
:101B0000000F1CD0C90701D0A56100E0A562C4F890
:101B100028C0C4F818C0A8F10108B8F1000F08D017
:101B2000C4F828C0C4F818C0A8F10108B8F1000F23
:101B3000F6D1A661C4F828C0C4F818C009E0A661AF
:101B4000C90701D0A56100E0A562C4F828C0C4F8A7
:101B500018C0C4F828C0C4F818C0A662C4F828C0C9
:101B6000C4F818C0A561000603D50A484068CAF841
:101B700008009AF80C0003E0C4F828C0C4F818C0A4
:101B8000401E411CF8D109F0FF00BDE8F0870000BD
:101B900054130020001000E02DE9F04F4FF0904565
:101BA0000127AF614FF0020CC5F828C0DFF8E482CE
:101BB000D8F8042013465B1EFDD1C5F818C01346A3
:101BC0005B1EFDD1AF62C5F828C013465B1EFDD178
:101BD000C5F818C013465B1EFDD1C5F828C01346D2
:101BE0005B1EFDD1C5F818C013465B1EFDD198F8E9
:101BF0001B4064B1C5F828C013465B1EFDD1C5F873
:101C000018C013465B1EFDD1641E002CF2D14308A0
:101C1000DB074FF0800601D0AE6100E0AE62C5F890
:101C200028C013465B1EFDD12B69C3F38014C5F891
:101C300018C013465B1EFDD164008308DB0701D08A
:101C4000AE6100E0AE62C5F828C013465B1EFDD150
:101C50002B69C3F38019C5F818C013465B1EFDD16C
:101C600044EA0904C308DB0701D0AE6100E0AE62BC
:101C7000C5F828C013465B1EFDD12B69C3F380193C
:101C8000C5F818C013465B1EFDD144EA8909B9F1B5
:101C9000010F0AD0AF61C5F828C01146491EFDD119
:101CA000C5F818C0521EFDD1C4E07A4C5FEA807AB4
:101CB000A37EE47EA3EB040865D500241F23C5F8AA
:101CC00028C09246BAF1010AFCD1D5F810A0CAF397
:101CD000801AC5F818C09346BBF1010BFCD144EA49
:101CE000CA7464085B1E002BE9D1A8F10108B8F1A1
:101CF000000F33D0E2462B46C5F828C09346BBF10F
:101D0000010BFCD1D3F810B0CBF3801BC3F818A0A3
:101D10009646BEF1010EFCD1A8F10108B8F1000F02
:101D200010D0C3F828A09646BEF1010EFCD1C3F82E
:101D300018A09646BEF1010EFCD1A8F10108B8F139
:101D4000000FEED19F61C3F828A09046B8F10108BA
:101D5000FCD1C3F818A0521EFDD10FE0A846AF6118
:101D6000E246C8F828C013465B1EFDD1D8F81030F3
:101D7000C3F3801BC8F818A0521EFDD144EACB72F1
:101D8000F1B30A6056E009681F24CB0701D0AE61A9
:101D900000E0AE62C5F828C013465B1EFDD1C5F851
:101DA00018C013465B1EFDD14908641E002CECD1FF
:101DB000A8F10108B8F1000F2CD0C90701D0AE611D
:101DC00000E0AE6264462B46C5F828C01146491EA5
:101DD000FDD19C611146491EFDD1A8F10108B8F161
:101DE000000F0CD09C621146491EFDD19C6111462A
:101DF000491EFDD1A8F10108B8F1000FF2D100E0B1
:101E000018E09F619C621146491EFDD19C61521EE3
:101E1000FDD10FE02B46AF61C90701D09E6100E004
:101E20009E626446C3F828C01146491EFDD19C61DC
:101E3000521EFDD1C5F828C0164A53681946491EDE
:101E4000FDD1C5F818C01946491EFDD1AF62C5F8CD
:101E500028C01946491EFDD1C5F818C01946491EAB
:101E6000FDD1AE61000602D50B4840689060107B42
:101E700009E0C5F828C01A46521EFDD1C5F818C0A1
:101E80001946491EFDD1401E411CF2D109F0FF0048
:101E9000BDE8F08F54130020001000E02DE9F04160
:101EA0004FF0904301259D6102249C62DFF84CC1F4
:101EB000DCF804100A46521EFDD19C610A46521EEF
:101EC000FDD19D629C620A46521EFDD19C610A466C
:101ED000521EFDD19C620A46521EFDD19C610A46EB
:101EE000521EFDD19CF81B60374656B19C620A46D3
:101EF000521EFDD19C610A46521EFDD1761E002E57
:101F0000F4D180269E629C620A46521EFDD19C61DD
:101F10000A46521EFDD19C620A46521EFDD19C61AA
:101F20000A46521EFDD19C620A46521EFDD19C619A
:101F30000A46521EFDD14FF01F08C20701D09E6114
:101F400000E09E629C620A46521EFDD19C610A46D8
:101F5000521EFDD14008A8F10108B8F1000FECD1E4
:101F60009CF81A20D21B521E2AB3C00701D09E61D2
:101F700000E09E629C620846401EFDD11F469C61A7
:101F80000846401EFDD1521E52B1BC620846401E9A
:101F9000FDD1BC610846401EFDD1521E002AF4D17D
:101FA000BD612246BC620846401EFDD1BA610846AA
:101FB000401EFDD10FE09D61C00701D09E6100E091
:101FC0009E6222461F469C620846401EFDD1BA61B1
:101FD0000846401EFDD19C620846401EFDD19C6112
:101FE0000846401EFDD19D629C620846401EFDD100
:101FF0009C61491EFDD19E61BDE8F0815413002013
:10200000014802F01FBB0000A80200207CB501219E
:10201000194800F09FFF18480121401C00F09AFF6A
:10202000684601F0EDF80225009500208DF80600C5
:102030004FF090466946304601F0ECF801240094D8
:102040006946304601F0E6F800956946304601F0F1
:10205000E1F800946946304601F0DCF880210091F7
:102060006946304601F0D6F8402100916946304675
:1020700001F0D0F87CBD000011001400F0B500F0B4
:102080003F03002B00D14023DFF88CC000064FF047
:1020900002064FF090451AD41CE00027082010E0FB
:1020A000AE62DCF804100C46641EFDD12C69C4F34A
:1020B0000004AE61491EFDD1790841EAC417401EF3
:1020C0005B1E08B1002BEBD1C74002F8017B002B4F
:1020D000E3D1F0BD10484FF0010C476818E011F84B
:1020E000012B082411E0D00702D0C5F818C001E088
:1020F000C5F828C0AE623846401EFDD1AE613846F4
:10210000401EFDD15208641E5B1E0CB1002BEAD1AB
:10211000002BE4D1F0BD000054130020034A527894
:10212000002A01D000F004B800F042B95413002096
:102130002DE9F0434FF090474FF00108C7F81880A1
:102140004FF0020CC7F828C0C7F818C0C20702D069
:10215000C7F8188001E0C7F82880C7F828C0C7F87A
:1021600018C003464208D40702D0C7F8188001E01F
:10217000C7F82880C7F828C0C7F818C013448208D9
:10218000D40702D0C7F8188001E0C7F82880C7F844
:1021900028C0C7F818C01344C208D40702D0C7F833
:1021A000188001E0C7F82880C7F828C0C7F818C011
:1021B0001A44D20702D0C7F8188001E0C7F8288077
:1021C000C7F828C0C7F818C0C7F82880C7F828C0C3
:1021D000C7F818C0C7F81880C7F828C0C7F818C0D3
:1021E0003A6822F003023A60DFF8BC9199F818309F
:1021F0001C4633B1C7F828C0C7F818C05B1E002BB7
:10220000F8D1C7F828C03A69C2F30002C7F818C06D
:10221000C7F828C03B69C3F30003C7F818C042EAF7
:102220004303C7F828C03A69C2F30002C7F818C0D0
:1022300043EA8202012A17D0022A7CD0042A7AD0EB
:10224000213434B1C7F828C0C7F818C0641E002C68
:10225000F8D1C7F82880386840F001003860C7F826
:102260001880D0B2BDE8F08383072CD50026002467
:102270002023C7F828C03D69C5F30005C7F818C07A
:102280002C44760846EAC5765B1E002BF1D1C7F8D0
:1022900028C03B69C7F818C05C40E30700D008229B
:1022A00001B10E6099F8181031B1C7F828C0C7F80D
:1022B00018C0491E0029F8D1C7F82880396841F0B4
:1022C000010139602BE034B1C7F828C0C7F818C045
:1022D000641E002CF8D1C7F828803B6843F0010346
:1022E0003B60096800242023CD0702D0C7F818807E
:1022F00001E0C7F82880C7F828C0C7F818C00C4408
:1023000049085B1E002BEFD1E10702D0C7F8188007
:1023100001E0C7F82880C7F828C0C7F818C0000631
:1023200003D522484068C9F8080099F80C0050B15C
:10233000C7F8288000E00AE0C7F828C0C7F818C02E
:10234000401E0028F6D1C7F81880D0B28AE799F865
:1023500019304BB1810707D52121C7F828C0C7F82C
:1023600018C0491E0029F8D134B1C7F828C0C7F8F1
:1023700018C0641E002CF8D1C7F82880396841F0D5
:10238000010139605BB1800709D4C7F8288021209A
:10239000C7F828C0C7F818C0401E0028F8D1C7F8F1
:1023A0001880D0B25EE7000054130020001000E057
:1023B0002DE9F04F00244FF090474FF00108C7F887
:1023C00018804FF0020CC7F828C0DFF88C93D9F8BA
:1023D000042013465B1EFDD1C7F818C013465B1ED0
:1023E000FDD1C30702D0C7F8188001E0C7F82880E4
:1023F000C7F828C013465B1EFDD1C7F818C01346A6
:102400005B1EFDD125184408E30702D0C7F81880E9
:1024100001E0C7F82880C7F828C013465B1EFDD12D
:10242000C7F818C013465B1EFDD125448408E30796
:1024300002D0C7F8188001E0C7F82880C7F828C084
:1024400013465B1EFDD1C7F818C013465B1EFDD1B5
:102450002544C408E30702D0C7F8188001E0C7F894
:102460002880C7F828C013465B1EFDD1C7F818C0E6
:1024700013465B1EFDD12B19DB0702D0C7F818806D
:1024800001E0C7F82880C7F828C013465B1EFDD1BD
:10249000C7F818C013465B1EFDD1C7F82880C7F8DF
:1024A00028C013465B1EFDD1C7F818C013465B1E3B
:1024B000FDD1C7F81880C7F828C013465B1EFDD1B0
:1024C000C7F818C013465B1EFDD13B6823F0030319
:1024D0003B6099F81840254664B1C7F828C01346F8
:1024E0005B1EFDD1C7F818C013465B1EFDD1641EEC
:1024F000002CF2D1C7F828C013465B1EFDD13B6902
:10250000C3F30004C7F818C013465B1EFDD1C7F81B
:1025100028C013465B1EFDD13B69C3F30006C7F814
:1025200018C013465B1EFDD144EA4604C7F828C014
:1025300013465B1EFDD13B69C3F30006C7F818C004
:1025400013465B1EFDD144EA8604012C1DD0022CEB
:102550007ED0042C7CD0213565B1C7F828C0104648
:10256000401EFDD1C7F818C01046401EFDD16D1E9B
:10257000002DF2D1C7F82880386840F0010038609B
:10258000C7F81880E0B2BDE8F08F830748D54FF058
:10259000000A00252023C7F828C01646761EFDD164
:1025A0003E69C6F30006C7F818C09346BBF1010B9D
:1025B000FCD135444FEA5A0A4AEAC67A5B1E002B20
:1025C000E9D13B46C7F828C0CE461646761EFDD157
:1025D0001E69C6F30006E346C3F818C0521EFDD1BB
:1025E0007540EA0700D0082409B1C1F800A09EF8A0
:1025F000182072B1DEF80450C3F828B02946491EED
:10260000FDD1C3F818B02946491EFDD1521E002A3B
:10261000F2D1C3F82880196841F0010119603FE048
:1026200065B1C7F828C013465B1EFDD1C7F818C0B6
:1026300013465B1EFDD16D1E002DF2D1C7F8288018
:102640003B6843F001033B6009680026202500E059
:1026500044E0CB0702D0C7F8188001E0C7F8288013
:10266000C7F828C013465B1EFDD1C7F818C0134633
:102670005B1EFDD10E4449086D1E002DE7D1F10708
:1026800002D0C7F8188001E0C7F8288063463D46AD
:10269000C7F828C01146491EFDD1AB61521EFDD1BD
:1026A000000603D52D484068C9F8080099F80C10B9
:1026B00081B1C7F82880D9F80420C7F828C010468F
:1026C000401EFDD1C7F818C01046401EFDD1491E5E
:1026D0000029F2D1C7F81880E0B254E799F8193010
:1026E0007BB181070DD52126C7F828C01146491EA8
:1026F000FDD1C7F818C01146491EFDD1761E002E27
:10270000F2D165B1C7F828C01146491EFDD1C7F8FE
:1027100018C01146491EFDD16D1E002DF2D1C7F81B
:102720002880396841F0010139608BB180070FD4EE
:10273000C7F828802121C7F828C01046401EFDD1C7
:10274000C7F818C01046401EFDD1491E0029F2D11D
:10275000C7F81880E0B216E754130020001000E01C
:10276000F0B500220023104C01274FF090464FF0A7
:10277000020C656814E013B911F8012B0823D40783
:1027800001D0B76100E0B762C6F828C02C46641ECD
:10279000FDD1C6F818C02C46641EFDD152085B1E40
:1027A000401E441CE7D1F0BD5413002002480168CC
:1027B000491C0160704700000000002011480168BA
:1027C00041F00101016001688907FCD5416821F0F1
:1027D00003014160416811F00C0FFBD101680A4A06
:1027E000114001600021416041F61071C1624FF457
:1027F000801101634FF41F01816004494FF00060B4
:102800000860704700100240FFFFF2FE08ED00E094
:1028100008B50121134800F09DFB0121124800F08A
:1028200099FB012000F028FC41F62C7000F094F98F
:102830004FF4FA5000F096F941F6547000F098F910
:102840000121022000F074F908480090084B002292
:102850000121084801F0B2FE07494FF0004008602E
:1028600008BD00000C0014001B001C0058010020D3
:102870004C020020A802002000E100E02DE9F04316
:1028800087B00121484800F065FB0121474800F06E
:1028900061FB01214FF4A01000F05CFB05A800F0E3
:1028A000AFFC02258DF81A500C2005904FF0904493
:1028B00005A9204600F0AEFC01220221204600F0CE
:1028C000DBFC01220321204600F0D6FCDFF8E0808B
:1028D00035220121404600F0E7FB1020ADF808004A
:1028E0003448019000248DF80F4001268DF80D60CA
:1028F000314F00978DF80E408DF80C40ADF80A402E
:102900008DF811508DF81040DFF8A490694609F158
:102910000809484600F00AFC0121484600F0BAFBCD
:1029200034220221404600F0BFFBADF808402148A8
:10293000803801908DF80F408DF80D6000978DF86C
:102940000E408DF80C408020ADF80A008DF8115033
:102950008DF81060164C69461C34204600F0E6FBEA
:102960000121204600F096FB3C1F002301224FF47A
:10297000E131204600F080FD0121204600F071FD8C
:102980000121204600F068FD0121204600F0E4FD11
:102990000121204600F0DBFD0121204600F066FD0C
:1029A00007B0BDE8F08300001100140011001C0006
:1029B00000000240141300200444004070B58179E7
:1029C00007291CD008291CD001224179D9B101293D
:1029D0001BD002291BD000240179D1B101291AD0C2
:1029E00002291AD0002372B601680D4D284600F066
:1029F00043FD2146284600F089FD62B670BD0022E5
:102A0000E3E70122E1E70024E6E70224E4E701240A
:102A1000E2E70023E7E70323E5E70223E3E700001B
:102A2000004400402DE9F0473B4DB5F852083B4FBC
:102A30004FF00008002842D0394800F030FBC0F1C8
:102A40008004384EDFF8E0907068211A402906D2E1
:102A5000844228D0D9F800103268914223D08442B1
:102A600000D28024211A402901D900F14004211A02
:102A7000A5F85018A5F85288B5F850282B490144FC
:102A80002A4888388246FDF728FCB5F85038524667
:102A90008321381D01F089FB04F07F007060D9F8B4
:102AA000000030600BE0B5F85008402807D1A5F8C9
:102AB000508800231A468321381D01F076FBB5F8B3
:102AC0009608002826D0164C143C204600F0E7FA61
:102AD00000281FD1A5F89688B5F8942813494439E1
:102AE0000E4601F1C400FDF73DFC0021204600F038
:102AF000D1FAB5F89418204600F0D4FA0121204606
:102B000000F0C8FA402303213246381DBDE8F047E3
:102B100001F0F9BABDE8F087FC090020A802002006
:102B20001C000240980200200000002094120020A7
:102B3000084A002808D0106840F0020010601068B1
:102B400061F3000010607047106820F00200106010
:102B5000F5E70000046C0040014908607047000080
:102B60000C6C00400149086070470000106C004088
:102B70000149086070470000146C004010B504461D
:102B80008121204601F094FA0121204601F090FABB
:102B90008221204601F08CFA8321204601F088FA38
:102BA0000321204601F084FA002010BD10B504482E
:102BB0004078202802D10348FFF700FF002010BD15
:102BC00088020020900200200020704700207047FB
:102BD00010B541F08000812802D0832807D102E09F
:102BE000FEF702FD03E003490120A1F8520800208E
:102BF00010BD0000FC09002010B50446402302224D
:102C00008121204601F065FA40230222012120465D
:102C100001F05FFA4023114A0121204601F073FAC6
:102C2000082303228221204601F053FA4023022286
:102C30008321204601F04DFA402302220321204641
:102C400001F047FA4023064A0321204601F05BFACF
:102C500004490120A1F85208002010BDAC05002055
:102C600050120020FC09002070B50C460546214694
:102C7000284601F0D9FB0146012C02D0032C10D1CB
:102C800009E00948FEF782FC4023074A0121284653
:102C900001F039FA05E00548A0F894180121A0F8E0
:102CA0009618002070BD0000AC050020FC09002033
:102CB00010B52C4A0B6853614B6893610A7812F087
:102CC000600205D0202A22D001F0C8F8002010BDF3
:102CD0004A78062AFAD14A882223B3EB122F09D167
:102CE000214AC988527E8A4200D30A461F4901F010
:102CF000A1F8EBE72123B3EB122FE7D1CA88092A09
:102D000000D909221849123101F094F8DEE74A7817
:102D10000B2A0FD008DC012A0CD0032A0AD0092A7A
:102D200008D00A2A06D1D1E7202A0ED0212A04D0C1
:102D3000222A12D001F092F8C8E7CA88072A00D3E5
:102D400007220B4901F076F8C0E7CA88072A00D3AA
:102D50000722074901F05AF8B8E748880549A1F861
:102D60000C08B3E7740200203800002004000020A3
:102D700090020020FC0900200020704702494A68A8
:102D800060F307124A6070470010024002494A6827
:102D900060F30A224A6070470010024002494A6804
:102DA00060F3CD224A60704700100240104A0528A7
:102DB00008D2DFE800F003080D121700106861F375
:102DC000000010607047106861F310401060704799
:102DD000106861F3186010607047106A61F30000BA
:102DE00010627047506A61F3000050627047000043
:102DF000001002402DE9F041044600F035F901468B
:102E00003C483D4D61B3012935D0022935D02060C1
:102E10006868C0F303103949095C2068C8406060E5
:102E20006968C1F30221354A183A515C20FA01F170
:102E3000E1606968C1F3C2210832515CC840A060FA
:102E40006968C1F300716A68C2F3813242EA8101A4
:102E50002A4A083A515CB0FBF1F02061BDE8F081EC
:102E6000696D890505D5296B890102D52448206043
:102E7000CEE72060CCE72060CAE76968C1F3004173
:102E8000EA6A002A1DDB6868C0F383406A68C2F3FF
:102E9000417252B90F2808D0801C51B1696889036A
:102EA0000BD5184948432060B2E700EB0210401CE4
:102EB000F3E7144948432060AAE70E4948432060DD
:102EC000A6E7EA6AC2F30312EB6AC3F30823EE6AC9
:102ED00006F007060B4F59B16968890300D53846DB
:102EE000A0FB0301B2400023FDF780F920608FE7CB
:102EF0003846F5E700127A0000100240AC4A00089C
:102F0000006CDC0200093D000146002001F01F03B7
:102F100001229A40034B03EB114109688A4300D117
:102F2000012070470010024002490A6B60F35962A9
:102F30000A6370470010024000B503460120FFF706
:102F4000F3FF0348416D63F34921416500BD000073
:102F50000010024010B500F01F030122064C9A40F9
:102F600004EB1040012903D001689143016010BDBA
:102F700001681143016010BD0010024030B500230C
:102F8000264A274C002815D0656845F480356560D1
:102F9000012814D0606840F4003060602148224D60
:102FA0001044A8422CD32148214D1044A8420CD2F1
:102FB000012325E0606820F480306060EEE71D4A60
:102FC000606820F400306060E8E71B481B4D104447
:102FD000A84201D2022313E019481A4D1044A84216
:102FE00001D203230CE01848184D1044A84201D226
:102FF000042305E016481044164A904200D20523E7
:10300000606861F3954060606068090961F35E7013
:103010006060E06A63F31A60E06230BD00093D0061
:10302000001002409F7DC4FFDFC810007FA7B0FFE3
:103030008F05100000127A006BCA88FF7BE507003D
:10304000EFE480FF0FA13F00D79411FF076C4F0002
:10305000CF28C2FEA7129F0002494A6860F301020E
:103060004A6070470010024002484068C0F3810087
:10307000704700000010024010B50446012C01D139
:10308000FFF75AFF0248416D64F30821416510BD06
:1030900000100240026861F300020260704740685D
:1030A00080B2704741607047D0F8A430DB0105D48E
:1030B000D0F8A43043F08073C0F8A430012911D0B7
:1030C000022915D0032919D004291DD0052921D0A2
:1030D000062925D0072904D150F8A41F62F317410F
:1030E0000160704750F8A01F62F30701016070474C
:1030F00050F8A01F62F30F210160704750F8A01F25
:1031000062F317410160704750F8A01F62F31F611E
:103110000160704750F8A41F62F307010160704717
:1031200050F8A41F62F30F210160704702684BF64C
:10313000EF731A40026002680B891A4302604B7CED
:10314000026863F30D320260CB7B026863F38B226B
:1031500002608B7B026863F3092202604B7B02688A
:1031600063F3C71202600B7B026863F3861202608E
:103170000B7C026863F3451202604A8942600A6868
:1031800082604968C16070470048704710010020A4
:1031900000487047E000002000487047D800002039
:1031A0000020704700487047080100200048704721
:1031B000E800002000487047F800002010B50B48D8
:1031C0000168001D0468001D00680844002809D03B
:1031D0000822074900F068F805490422103120460A
:1031E00000F062F802481A3810BD0000E8F7FF1F2F
:1031F0001A01002000487047F000002081617047EC
:103200004FF6FF710160002181710171417101214F
:10321000C1717047F0B500220B889BB229E0DC0732
:1032200024D0066854000325A540AE4306608E797D
:103230000768A6403E430660466801279740BE43A4
:10324000466046680F7997403E4346608668AE43C5
:103250008660CE798768A6403E438660C668AE43E6
:10326000C6604D79A540C4682543C5605B08521C03
:1032700092B2002BD3D1F0BD10B54B07DB0E9A40B4
:10328000CC084FF00F0101FA03F106D0436A8B43DB
:103290004362416A1143416210BD036A8B4303627A
:1032A000016A1143016210BDF0B500230A253026E2
:1032B0003727002411E0B5EB107F04D906EB107C12
:1032C00001F813C003E007EB107C01F813C001EB19
:1032D000430C8CF8014000015B1C9342EBDBF0BD1A
:1032E00000F024F8FEF7BCF8FFF7C8FAFFF790FAF1
:1032F0000C484FF47A710068B0FBF1F0401EB0F159
:10330000807F09D24FF0E0214861074AF020107019
:10331000002088610720086101F0ACF8FFF782FB0C
:10332000FAE70000A402002023ED00E010B51249E6
:103330004FF4A970086017210020FFF71FFE01213C
:103340000220FFF733FD1920FFF7DEFD0128FAD137
:103350000020FFF713FD0020FFF718FD0020FFF706
:103360001DFD0220FFF778FEFFF77EFE0228FBD14D
:10337000BDE8104000F002B8002002402DE9F04105
:10338000FFF772FE2E492F4D2F4C70B1012817D038
:10339000022817D021606868C0F303102B49085C2D
:1033A0002168C1402160BDE8F081686D800505D5C8
:1033B000286B800102D526482060ECE72160EAE70F
:1033C0002160E8E76868C0F30043E86A00281DDB75
:1033D0006868C0F383406968C1F3417151B90F282F
:1033E00008D0801C53B1696889030BD5194948433B
:1033F0002060D0E700EB0110401CF3E7154948437B
:103400002060C8E70E4948432060C4E7E86AC0F37B
:103410000312E86AC0F30820EE6A06F007060D4FB3
:103420005BB16B689B0300D53946A1FB0001B2403C
:103430000023FCF7DBFE2060ADE73946F5E700002E
:1034400000127A0000100240A4020020BC4A0008CA
:10345000006CDC0200093D00426961F386124261A2
:103460007047426961F3C71242617047C26861F3F5
:103470004D32C26070470000F0B585B004460F467B
:1034800015461E466846FFF7B5FC1F48844201D129
:10349000029800E0039800EB80004000B0FBF7F0DA
:1034A0000A21B0FBF1F201FB1202052A02D2B0FBA5
:1034B000F1F002E0B0FBF1F0401CA16860F30F01F5
:1034C000A1607DB1012D16D0E06820F08050E06051
:1034D000E06840F48050E060206966F30D302061C0
:1034E00005B0F0BDE06840F08050E060E06820F496
:1034F0008050E060F0E7E06820F08050E060E06835
:1035000020F48050E060E7E70038014000290CD04B
:10351000012913D0022907D1C16841F40071C160AB
:10352000C16841F48061C1607047C16821F40071D5
:10353000C160C16821F48061C1607047C16821F435
:103540000071C160C16841F48061C1607047C268A8
:1035500061F38202C2607047C26861F3C302C26055
:103560007047D0F8041821F00201C0F80418704721
:1035700000F53D70017041720022C2724273402218
:1035800082800822C2704FF4A072C280A0F53D7004
:10359000012902D1022180F8FC12012180F80113D7
:1035A00000207047D0F8041841F00201C0F8041858
:1035B0007047D0F800196FF30A01C0F80019D0F86D
:1035C000041821F48071C0F80418704700F53060C9
:1035D000002101610169012262F3DC41016101699D
:1035E0006FF3120118310161016941F0C0410161BD
:1035F00070478B780A78002B00EB421214D0D2F877
:10360000003B23F40013C2F8003BCA78032A01D020
:10361000022A08D1097800EB4110D0F8001B41F0D4
:103620008051C0F8001B7047D2F8003923F4001312
:10363000C2F80039CA78032A01D0022AF3D10978E6
:1036400000EB4110D0F8001941F08051C0F800198A
:10365000704710B50B788C7801229A40002C0FD05F
:10366000D0F81C3823EA0242C0F81C28097800EB85
:103670004110D0F8001B21F40041C0F8001B10BD20
:10368000D0F81C389343C0F81C38097800EB41107F
:10369000D0F8001921F40041C0F8001910BD10B590
:1036A0000021002301EB410202EBC10200EB820288
:1036B000117351739373536113625362491CC9B2FE
:1036C0000829EFD30021012401EB410202EBC102E2
:1036D00000EB820202F5B672117051709470936023
:1036E00053619361491CC9B20829EDD310BD00EBA9
:1036F0004110C0F808297047D0F81028D0F83438A5
:10370000CB4003F0010342EAC31200EB4110D0F8B2
:1037100008091040704730B500220B78002B0ED1FD
:103720008B68402B0BD0202B04D0102B04D0082BFF
:1037300004D004E0012202E0022200E003220D781E
:103740008C780123AB406CB3D0F81C4844EA0343A7
:10375000C0F81C380B78F3B300EB43120C89D2F895
:10376000003B64F30A03C2F8003B0A78CC7800EB14
:103770004212D2F8003B64F39343C2F8003B0A784C
:1037800000EB4212D2F8003B43F08053C2F8003BFA
:10379000097800EB4110D0F8001B41F40041C0F85B
:1037A000001B30BDD0F81C481C43C0F81C480B78E7
:1037B00083B300EB43120C89D2F8003964F30A0397
:1037C000C2F800390A78CC7800EB4212D2F80039FE
:1037D00064F3934300E025E0C2F800390A7800EB77
:1037E0004213D3F8004962F39954C3F800490A78A8
:1037F00000EB4212D2F8003943F08053C2F800398E
:10380000097800EB4110D0F8001941F40041C0F8EC
:10381000001930BDFFE7D0F8003962F30A03C0F8A1
:103820000039CFE7D0F8003B62F30A03C0F8003B51
:103830009BE700EB4110C0F8082B704700EB4111EB
:10384000D1F8081BD0F81408084070478B780A7824
:10385000002B00EB421213D0D2F8003B002B05DB0B
:10386000D2F8003B23F08043C2F8003B097800EB1C
:103870004110D0F8001B41F40011C0F8001B704744
:10388000D2F80039002B05DBD2F8003923F0804351
:10389000C2F80039097800EB4110D0F8001941F462
:1038A0000011C0F8001970470021026942F01002AF
:1038B0000261054A03E00B46491C934202D80369A2
:1038C000DB06F8D470470000400D030000220369B6
:1038D00061F38A130361016941F020010161054927
:1038E00003E01346521C8B4202D803699B06F8D4AE
:1038F00070470000400D0300D0F81818D0F81C08DD
:1039000089B208407047D0F81818D0F81C08084051
:10391000000C7047416170474169806908407047F9
:1039200010B50446204600F00FF8A06B40F480303C
:10393000A06310BD012A03D082698A438261704767
:1039400082690A438261704700210C4A03E00B46FA
:10395000491C934202D80369002BF8DA002103695D
:1039600043F00103036103E00B46491C934202D874
:103970000369DB07F8D1012070470000400D030008
:103980004FF0A0407047002907D1C26822F00052D2
:10399000C260C26842F08042C260012907D1C26899
:1039A00022F08042C260C26842F00052C260022926
:1039B00007D1C16821F08041C160C16821F0005188
:1039C000C1607047816821F00101816070478168A2
:1039D00041F0010181607047D0F8001E21F0010123
:1039E000C0F8001E704710B5DB1C9B08002200F5D4
:1039F000805002E0046810C1521C9A42FAD310BDF4
:103A0000D0F8002861F30A12C0F80028704741621C
:103A1000704730B50023446A002904D0856A04EB5E
:103A20001544491E0BE044EA0241816230BD00EBBF
:103A30008305D5F8045104EB15445B1CDBB28B42C3
:103A4000F5DB00EB810044EA0242C0F8042130BDFE
:103A5000D0F8001E41F00101C0F8001E7047D0F8F8
:103A6000080800F0010070472DE9F0470E4607688E
:103A700006EB460101EBC60100EB81040C34D4E9EE
:103A80000601451AA068A84200D20546E81C4FEA84
:103A9000900907EB461813E0D51AA268AA4200D293
:103AA0001546E81C4FEA9009ABB2B2B238466169DC
:103AB00000F01CF8606928446061E0692844E06116
:103AC000D8F8180980B2484505D9D4E906239342AD
:103AD00001D2002AE0D1002D06D1D7F83408012107
:103AE000B1408843C7F83408BDE8F08710B5DB1C47
:103AF0009C08002300EB023000F5805002E004C96E
:103B000002605B1CA342FAD310BD70B504460025C9
:103B100004F5337194F8E402022806D0032804D097
:103B2000204600F09BF9284670BD48880128FAD14C
:103B3000002084F8E702D4F8EC0220F00200C4F878
:103B4000EC026068826820469047204600F07EF9CB
:103B5000E9E710B502680B0601F07F0101EB4104B3
:103B600004EBC10100EB810401D50C3401E004F544
:103B7000B67421461046FFF73CFD0020607310BD6F
:103B80000068FFF7EEBC70B5044601F07F0000EB63
:103B9000400202EBC00004EB80020C3200290BD083
:103BA00060684269002A45D094F8E402032841D1B4
:103BB0002046BDE87040104794F8E002022839D151
:103BC000516A906881420DD9081A50629168884202
:103BD00000D3084683B252692046BDE870400021F8
:103BE00000F0E3BA116A814216D1916A814213D37F
:103BF000B4F8E20281420FD20025156200231A4672
:103C00001946204600F0D1FA29462046BDE870400A
:103C100000231A4600F077BA6068C16829B194F8A9
:103C2000E402032801D1204688472046BDE87040C1
:103C300000F0F8B870BD00002DE9F0410646316093
:103C40000C4604F50065012086F8E402002786F89A
:103C5000E6727260B360304600F05AF93046FFF702
:103C60001EFD2046FFF7AEFE2046FFF759FE00215D
:103C70002046FFF788FE3068FFF7AEFE286820F484
:103C8000C0502860286840F00300286010212046BA
:103C9000FFF71CFE2046FFF707FE781EA861EF61C4
:103CA0002F616F61002004EB8001C1F80471401C9A
:103CB0000828F8D3304600F0F3FA0020FF2104EB87
:103CC000401202F510621368002B09DA17601368BE
:103CD00043F080431360136843F00063136000E017
:103CE000176017619160401C0828E8D3002004EB9E
:103CF000401202F530621368002B09DA176013686E
:103D000043F080431360136843F00063136000E0E6
:103D1000176017619160401C0828E8D3286940F4B7
:103D200080702861A7616FF0804060610548A061E4
:103D30003046FFF725FF2046FFF749FE0020BDE88B
:103D4000F08100001C383C8010B5044601F07F0073
:103D500000EB400202EBC00004EB800202F5B672F9
:103D600000290BD060688269002A26D094F8E4020A
:103D7000032822D12046BDE81040104794F8E00205
:103D800003281AD19368506A98420CD9C01A50621D
:103D90009368984200D3184683B252692046BDE822
:103DA000104000F0B0B96068016909B12046884749
:103DB0002046BDE8104000F049B810BD10B50446DB
:103DC00004F5357104F5337000F012FE012084F81B
:103DD000E002B4F8D202A4F8E20294F8CC0210F0A7
:103DE0001F0008D001280BD002280ED12046BDE8C4
:103DF000104000F090B82046BDE8104000F03AB8FE
:103E00002046BDE8104000F003BC10BD00F5B673BD
:103E10009A625A62032380F8E03213460A46002170
:103E200000F071B9052180F8E01200231A46194606
:103E300000F069B900F10C039A625A62022380F81B
:103E4000E03213460A46002100F0AFB9042180F8A1
:103E5000E01200231A46194600F0A7B910B504462F
:103E60000021204600F0ADFD2046BDE81040802135
:103E700000F0A7BD10B5002400F533710A78C2F335
:103E80004112022A0CD0012A21D090F8CD120A2921
:103E900037D2DFE801F021243627362A2D36303399
:103EA0004A78342A02D10A79072A03D0FFF7D6FFCD
:103EB000204610BD154AC988137A527A43EA022275
:103EC0008A4200D90A461149FFF7B4FFF0E7426879
:103ED00092689047204610BD00F0B1FA13E0FFF75A
:103EE00014FE10E000F05AFD0DE000F0DDFC0AE0E9
:103EF00000F02DFA07E000F007FA04E000F0F8FC0B
:103F000001E0FFF7ABFF204610BD0000A401002038
:103F10000068FFF747BB2DE9F0410546002705F58E
:103F2000337634793078C0F34110012804D16868C1
:103F30003146826828469047707848B101283CD0C5
:103F400003285FD02846FFF789FF3846BDE8F08197
:103F500095F8E402022805D003280AD02846FFF786
:103F60007DFFF2E76006F0D02146284600F029FDEB
:103F7000EBE7200609D504F07F0000EB400101EBE0
:103F8000C00005EB80010C3109E004F07F0000EB7C
:103F9000400101EBC00005EB800101F5B671487BE3
:103FA000012807D000200861022210312846FFF7BF
:103FB00041FFCAE701200861F6E795F8E40202280C
:103FC00005D003280CD02846FFF748FFBDE7002C9A
:103FD000BBD0802CB9D02146284600F0F2FCB4E7D3
:103FE00070880028B1D1600608D021462846FFF726
:103FF000B0FD686831468268284690472846FFF73A
:1040000025FFA2E795F8E402022805D003280CD08A
:104010002846FFF723FF98E7002C96D0802C94D0F9
:104020002146284600F0CDFC8FE7708830B92CB1CE
:10403000802C03D02146284600F0C3FC6868314636
:104040008268284690472846FFF700FF7DE710B5B5
:1040500004462068FFF703FD012804D12068BDE86D
:104060001040FFF7F5BC10BD70B504462568284622
:10407000FFF79FFAE86820F4705000F5A050E86060
:10408000002240231146204600F023F8402300225E
:104090008021204600F01DF8012084F8E4026068C9
:1040A0004168002903D02046BDE87040084770BD34
:1040B0000A0601F07F0101EB410303EBC10100EBB4
:1040C000810101D50C3101E001F5B6710068FFF7FF
:1040D000C0BAF0B404680D0601F07F0101EB41069F
:1040E00006EBC10100EB810104D401F5B67101209A
:1040F000887002E00C31002088708B60CA70204606
:10410000F0BCFFF708BB70B5056801F07F0404EB55
:10411000440606EBC40400EB840404F5B67420786E
:1041200005EB401000F5306005F500656261A361A4
:104130000022E2614A0601D1A268A261A2699AB195
:10414000490611D0A1680A44521EB2FBF1F203697C
:10415000514361F312030361016962F3DC410161C0
:10416000E17801290BD012E0A268016962F3120123
:1041700001610169012262F3DC410161F0E7A96894
:10418000090AC9070CD0016841F08051016001683B
:1041900041F080610160016841F00041016070BD43
:1041A000016841F000510160F1E7F0B4054628686C
:1041B00001F07F0404EB440606EBC40405EB840520
:1041C0000C352C7800EB441404F5106400F50066FF
:1041D0006A61AB610022EA61AA690123002A12D058
:1041E000490619D0A96857187F1EB7FBF1F1276956
:1041F00062F312072761226961F3DC422261E978E8
:10420000012919D01EE0216963F3DC412161216994
:104210006FF31201216115E0A9688A4200D9A961F2
:10422000AA69216962F312012161216963F3DC410A
:104230002161A969296205E0216921F0C04101F1EC
:1042400000512161E978012906D0A96921B1716B7A
:104250002A78934019437163E978012907D1B1683D
:10426000090AC90715D0216841F0805121602168F1
:1042700041F080612160216841F000412160E978CE
:1042800001290BD1298B2A788BB26969F0BCFFF721
:104290002DBC216841F000512160E8E7F0BC704777
:1042A00010B50468B4F1A04F2DD180212046FFF74E
:1042B000AEFB182200212046FFF7ABFB14220121A0
:1042C0002046FFF7A6FB142202212046FFF7A1FBA0
:1042D000142203212046FFF79CFB142204212046D0
:1042E000FFF797FB142205212046FFF792FB1422CB
:1042F00006212046FFF78DFB20461422BDE8104022
:104300000721FFF786BB10BD10B5002400F53371FF
:10431000C988012902D0FFF7A1FD07E090F8E41257
:10432000022905D003290CD0FFF798FD204610BDC7
:10433000002180F8E812012200F53A71FFF77AFDBA
:10434000F4E7012200F2E921FFF774FDEEE770B512
:10435000054600260024B5F8CE12080A06284CD0DF
:1043600006DC01280DD0022810D0032804D116E065
:10437000072854D00F280ED02846FFF76FFD30468F
:1043800070BDA86800688047044639E0A868806866
:104390008047044634E0FEF7F7FE044630E0C8B23A
:1043A000062822D2DFE800F003080D12171CA868C7
:1043B00000698047044623E0A868406980470446B6
:1043C0001EE0A86880698047044619E0A868C069B3
:1043D0008047044614E0A868406A804704460FE01E
:1043E000A868006A804704460AE0686805F53371EA
:1043F000826828469047304670BD2846FFF72EFD5C
:104400005CB122884AB1B5F8D20230B1824200D301
:10441000024628466168FFF70DFD304670BD28460C
:10442000FFF71CFD304670BD01F07F0101EB41023A
:1044300002EBC10100EB8100D0F88801704710B594
:10444000002490F8E412022905D0032903D0FFF7D5
:1044500005FD204610BD90F8E71229B1D0F8EC1206
:1044600041F00201C0F8EC12022200F53B71FFF7A7
:10447000E1FCEEE770B5214CA1686068814201D192
:104480006078B8B31E4DE068A26805EB8011A5F511
:10449000007000EB8210FCF7D5FBE26805F50071B7
:1044A00021F81200A068401C082800D10020A0605C
:1044B000A268636800209A4200D1607022785AB1E5
:1044C0002070E06831F81030E068812105EB80123F
:1044D0000C48FFF76AFE0BE0E068401C082800D19A
:1044E0000020E060E0682169884201D10120A070CD
:1044F000012070BDFFE70020FBE7000074020020F0
:10450000EC070020AC02002041680A6A002A01D0B2
:1045100005211047704741680A6A002A01D0062128
:10452000104770472DE9F0418046D8F8007000250B
:104530003846FFF7E1F906463CE0F00738D0294657
:104540003846FFF7D9F80446E0070FD0D7F834080B
:104550000121A9408843C7F834080122294638467A
:10456000FFF7C5F8E9B24046FFF70DFB200704D579
:10457000082229463846FFF7BAF8E00604D510228B
:1045800029463846FFF7B3F8600604D5402229468D
:104590003846FFF7ACF8A00704D502222946384672
:1045A000FFF7A5F8200603D529464046FFF75CFA39
:1045B0006D1C7608002EC0D1BDE8F0812DE9F843CE
:1045C0000446089F884610461E460025FFF7D8F986
:1045D000206041462046FEF7CBFF94F8FF0220B151
:1045E0002068816B41F48011816394F8010320B14C
:1045F0002068816B41F400118163CDF800803B4657
:104600003246201D2168FFF717FB2846BDE8F883D6
:1046100070B50446002604F533710D4694F8E402A3
:10462000032804D02046FFF719FC304670BD6068AF
:10463000826820469047E8880028F6D12046FFF798
:1046400005FCF2E770B50568061D2846FFF764F91A
:1046500004466869C0075BD1A00703D5022128463C
:10466000FFF758F9600302D53046FFF75BFF2003E0
:1046700002D5304600F04DF8E00407D5304600F092
:104680008AF84FF480512846FFF744F9200706D5F1
:10469000304600F0C1F908212846FFF73BF9A00495
:1046A00007D53046FFF7E0FC4FF400512846FFF7EE
:1046B00031F9E00602D5304600F0BCF8E00207D53B
:1046C0003046FFF721FF4FF480112846FFF722F90B
:1046D000A00207D53046FFF71EFF4FF40011284611
:1046E000FFF718F9002C07DA304600F0B6F94FF062
:1046F00000412846FFF70EF9200509D5304600F0A5
:1047000091F92846BDE870404FF40061FFF702B907
:1047100070BD2DE9F0410746D7F8008000244046DF
:10472000FFF7F1F8054632E0E8072ED02146404673
:10473000FFF784F80646F00708D0012221464046DC
:10474000FFF777F8E1B23846FFF7FEFA300715D5E4
:10475000082221464046FFF76CF8E1B23846FFF7E1
:104760002DFB97F8E61249B13868D0F8002861F3BC
:104770000A12C0F80028002087F8E602F00604D5E7
:10478000102221464046FFF754F8641C6D08002DA6
:10479000CAD1BDE8F0812DE9F04107463E6806F533
:1047A00000640025606820F0010060603846FFF773
:1047B00077FD10213046FFF789F8FF2006EB451101
:1047C000C1F80809C1F8080B6D1C082DF6D34FF08D
:1047D000FF30A0614FF00110E061606940F001001E
:1047E0006061606940F002006061606940F008004B
:1047F0006061206940F001002061206940F0020002
:104800002061206940F00800206100213046FFF758
:10481000F7F83046FEF7DAFE012087F8E402786800
:10482000026A002A04D03846BDE8F0410121104751
:10483000BDE8F0812DE9F0410646376800221021DD
:104840003846FFF777F83A6AC2F30A15C2F34340D5
:1048500002F00F0202EB420101EBC20106EB810400
:1048600004F5B674022802D006280DD015E0A5B1D3
:10487000ABB238466169FFF7B6F8606928446061F9
:10488000E0692844E06108E0ABB206F535713846CE
:10489000FFF7A9F8E0692844E0613846BDE8F04137
:1048A00001221021FFF746B810B5002400F533713E
:1048B0008A88002A01D1CA881AB1FFF7CFFA2046A8
:1048C00010BD897801F07F0190F8E422032A06D018
:1048D00080F8E61231B1022180F8E41205E0FFF71A
:1048E000BDFAECE7012180F8E412FFF7AFFAE6E742
:1048F00070B50446002504F53371274E8878307072
:104900008A88002A01D1C98821B12046FFF7A6FA7A
:10491000284670BD94F8E412022905D0032915D069
:104920002046FFF79BFAF3E760B184F8E902032021
:1049300084F8E40260680168204688472046FFF753
:1049400085FAE5E72046FFF781FAE1E790B194F8B0
:10495000E91281421BD1606841682046884730785F
:1049600084F8E90260680168204688472046FFF71E
:104970006DFACDE7022184F8E41284F8E902606858
:104980004168204688472046FFF760FAC0E7204686
:10499000FFF75CFABCE70000A102002070B50446F6
:1049A000002504F533714888012808D184F8E7020E
:1049B00060688268204690472046FFF747FA2846FD
:1049C00070BD10B502680B0601F07F0101EB4104D8
:1049D00004EBC10100EB810401D50C3401E004F5C6
:1049E000B67421461046FEF731FF0120607310BDFA
:1049F0000A7802704A7842708A78CB7802EB0322F8
:104A000042800A794B7902EB032282808A79C97944
:104A100002EB0121C18070474168C969002900D0BB
:104A20000847704710B504462068D0F80808C0074A
:104A300012D094F8E40284F8E502042084F8E40239
:104A40002046FFF704FB6068026A002A04D0204673
:104A5000BDE810400221104710BD10B50446206883
:104A6000D0F8041821F00101C0F804182068FEF7FE
:104A7000B3FF94F8E50284F8E4026068026A002A51
:104A800004D02046BDE810400321104710BD322E4F
:104A9000312E30000000000001020304000000007D
:104AA0000102030402040608020C081000000000C2
:104AB00000000000010203040607080900000000CE
:104AC000000000000102030406070809EC4A000880
:104AD00000000020A80200000C010008C44C0008DF
:104AE000A8020020502300006801000841120610AF
:104AF0000BFF0901A10119012940151326FF1675A5
:104B000008954081290F129132C035120101021F10
:104B1000403C2E2170100C23030114090262290865
:104B2000246409042302FF170507050102402D0133
:104B3000070581071008080B01020202011409048D
:104B400001190A12011305241610010524011D0282
:104B50000424020E10090601020705820308150A43
:104B600009040233020A1C0705833B19072A0307BD
:104B70002110080403090412035812491256124E58
:104B800012311239123832371A24141256122D12D9
:104B90004C1269126E126B12201243124D1A5328D6
:104BA0001A53161244124112502A1228213320623D
:104BB0001A380819A6111A9C0829181AA008191CD5
:104BC000111AB408321A4B1801101A340832211A7B
:104BD00080081C1A03307212321233123412351A42
:104BE00036781A388012410A2542801399311B0801
:104BF000A1041A9104411AAD081AF5041AB5041A51
:104C0000BD045AA51814050F2115011C100520110B
:104C1000DF60DDD88945C74C9CD2659D9E648A9F24
:104C20001C0306A67D31520A290F12083A02C81247
:104C30001412032E57494E55538F711280120412CD
:104C4000011A288012651A769A1A63081A49A01A5E
:104C50007408127212663A611212471A55163244DB
:104C6000124E1A7BB81A44D21A33041A35B61A44B3
:104C7000BE1A32E629101A2D7B1A36021A330A1A86
:104C800041021A330C122D3A310C3A451C290412F8
:104C9000331A37021236527D13F92B1B087D041389
:104CA000B12C1B08C9081AAD041AD1041A691013D3
:104CB000792D1B08CD0C41021C012AC21E3927A1E7
:044CC00013127A0051
:04000005080000D11E
:00000001FF
